:020000040000FA
:100000008316031300308600F03087003D202E2039
:100010001E2015200C20072803178312103091078B
:1000200021208312031386000800212012081002E9
:10003000031D1B281D28910A152808000030910077
:1000400008008312031711088D0083168C130C14FB
:100050000C18282883120C0892000800831203133E
:1000600007080317831290000310900C0310900CE4
:100070000310900C0310900C080083120317053036
:100080009100212005301202031D4D281E309100E1
:100090002120673012020319F02800308D00003053
:1000A0008C00F12001308D0001308C00F1200230F5
:1000B0008D0002308C00F12003308D0003308C0065
:1000C000F12004308D0004308C00F12005308D00CB
:1000D00005308C00F12006308D0006308C00F120B8
:1000E00007308D0007308C00F12008308D0008307B
:1000F0008C00F12009308D0009308C00F1200A308D
:100100008D000A308C00F1200B308D000B308C00FC
:10011000F1200C308D000C308C00F1200D308D0062
:100120000D308C00F1200E308D000E308C00F1204F
:100130000F308D000F308C00F12010308D00FC301E
:100140008C00F12011308D0060308C00F1201230D5
:100150008D00DA308C00F12013308D00F2308C00ED
:10016000F12014308D0066308C00F12015308D00A8
:10017000B6308C00F12016308D00BE308C00F1209E
:1001800017308D00E0308C00F12018308D00FE30EB
:100190008C00F12019308D00F6308C00F1201A30DF
:1001A0008D00FD308C00F1201B308D0061308C0003
:1001B000F1201C308D00DB308C00F1201D308D00D3
:1001C000F3308C00F1201E308D0067308C00F12060
:1001D0001F308D00B7308C00F120831603170C11EF
:1001E0000800831603170C1555308D00AA308D00BA
:0E01F0008C148C18F9280C12831203170800C7
:02400E00F13F80
:00000001FF
